:100000000C94CD000C94F5000C94F5000C94F500C4
:100010000C94F5000C94F5000C94F5000C94F5008C
:100020000C94F5000C94F5000C94F5000C94FB0C6A
:100030000C942F110C94F5000C94F5000C94F50021
:100040000C947F140C94F5000C948B160C94F50012
:100050000C94F5000C94F5000C94F5000C94F5004C
:100060000C94F5000C94F500746F6F206D616E793F
:10007000206F70656E2066696C6573006261642034
:10008000696E707574005941414B00594545454BA7
:100090000053616D706C65207261746520746F6FC0
:1000A0002068696768210000436F6D707265737323
:1000B000696F6E206E6F7420737570706F727465E7
:1000C00064006661696C656420746F2067657420E4
:1000D0006E657720636C7573746572002021212131
:1000E0002000203F3F3F200046696C657320666F0B
:1000F000756E643A0046696C657320666F756E6450
:100100003A00436F756C646E2774206F70656E20C3
:1001100064697200436F756C646E2774206F70653C
:100120006E2066696C65737973004E6F2070617222
:10013000746974696F6E21004361726420696E692D
:10014000742E206661696C65642100000024272AF2
:10015000000025282B00002326290404040404049D
:100160000404020202020202030303030303010266
:100170000408102040800102040810200102040835
:100180001020000000070002010000030406000028
:100190000000000000007911D71211241FBECFEF1C
:1001A000D4E0DEBFCDBF11E0A0E0B1E0E4E2FFE2C9
:1001B00002C005900D92A632B107D9F714E0A6E26D
:1001C000B1E001C01D92A637B107E1F711E0CAE91D
:1001D000D1E004C02297FE010E948C17C639D107D6
:1001E000C9F70E94D0120C9490170C940000089547
:1001F0000895CB010E941B030895FC018481958121
:100200000E94AD040895EF92FF920F931F93CF9336
:10021000DF93EB018A0179010BC0B801C7010E948D
:10022000C816009729F4CE010E94AD0481E006C0F3
:10023000B701CE010E94B604882379F7DF91CF91F0
:100240001F910F91FF90EF900895EF92FF920F93FF
:100250001F93DF93CF93CDB7DEB768970FB6F894AF
:10026000DEBF0FBECDBF8C017E010894E11CF11CE6
:1002700097010E940301882319F420E030E005C0B3
:10028000B701C8010E948F089C01C90168960FB68A
:10029000F894DEBF0FBECDBFCF91DF911F910F91BC
:1002A000FF90EF900895FC01AB016481758182811C
:1002B00093810E9425010895EF92FF920F931F935F
:1002C000DF93CF93CDB7DEB768970FB6F894DEBF54
:1002D0000FBECDBF8B017E010894E11CF11CB7015C
:1002E000FC01848195810E94B604882349F04CE08A
:1002F00050E0B701C8010E94DF16F801148681E0C2
:1003000068960FB6F894DEBF0FBECDBFCF91DF91D8
:100310001F910F91FF90EF900895FC0184819581CA
:100320000E94A7040895EF92FF920F931F93DF930B
:10033000CF93CDB7DEB768970FB6F894DEBF0FBE88
:10034000CDBF8C017E010894E11CF11CB701FC01BA
:10035000828193810E945905B701F80182819381BE
:100360000E944007F8019583848320E0892B09F0DF
:1003700021E0822F68960FB6F894DEBF0FBECDBF86
:10038000CF91DF911F910F91FF90EF9008950F9300
:100390001F938C01FC01808191810E946A05F80104
:1003A0009383828320E0892B09F021E0822F1F9123
:1003B0000F9108950F93CF93DF93EC0100E020E0BD
:1003C00030E040E050E06CE17BE082E69AE00E94A1
:1003D000D60899838883892B69F40FEF20E030E0F9
:1003E00040E050E06CE17BE082E69AE00E94D608B3
:1003F0009983888320E088819981892B09F021E005
:10040000822FDF91CF910F9108950E940C0A0895D9
:10041000FC01009711F0118210820895DC018C918B
:10042000853E39F1882329F1F901208131818281CA
:1004300093812817390799F444835583668377831A
:100440001B968C911B978F3011F080E205C08C9128
:100450008295880F807E805E808780E008951B965D
:100460008C918F3031F02F5F3F4F3183208381E0BB
:10047000089581E008950F931F93CF93DF938C012C
:10048000FC018081853E09F48CC0882309F489C071
:10049000E9018C899D89AE89BF890097A105B105C5
:1004A00021F44C8B5D8B6E8B7F8B209709F479C088
:1004B0000115110509F475C0F8018081882309F43C
:1004C00070C083858F3011F481E06CC0A801D80121
:1004D00080E090E0282F3C91303251F0FE01E80F8F
:1004E000F91F30832F5F019611968830910591F79F
:1004F0008881853011F485EE8883F801808580320B
:10050000B1F0FE01E20FF11D8EE28083822F8F5F3A
:100510002C5FFA019085903249F0FE01E80FF11D41
:1005200090838F5F4F5F5F4F821799F7282FFE01EF
:10053000E20FF11D1082F80183858D87938D80E095
:10054000228D30E0822B932B9F878E87258D30E084
:1005500040E050E0542F432F322F2227868D90E029
:10056000A0E0B0E0DC0199278827282B392B4A2B03
:100570005B2B848D90E0A0E0B0E0282B392B4A2B38
:100580005B2B878D90E0A0E0B0E0B82FAA279927D9
:100590008827282B392B4A2B5B2B288B398B4A8BAE
:1005A0005B8B80E0DF91CF911F910F910895DF93D6
:1005B000CF9300D0CDB7DEB7DC010097A1F1623058
:1005C000710588F1ED91FC911197660F771F80E01E
:1005D00090E016962D913D914D915C911997620F87
:1005E000731F841F951F0190F081E02D22E030E001
:1005F000AE014F5F5F4F09958823A9F09A8180E093
:10060000298130E0282B392B2115310571F08FEF2E
:10061000273F380741F0C9014096079720F08FEF38
:10062000283F380710F020E030E0C9010F900F900C
:10063000CF91DF910895FC01009711F01182108293
:1006400008952F923F924F925F926F927F928F9276
:100650009F92AF92BF92CF92DF92EF92FF920F9351
:100660001F93DF93CF93CDB7DEB72C970FB6F894D7
:10067000DEBF0FBECDBF3C0178876F835A874987A5
:10068000009709F402C1672B09F4FFC0452B09F458
:10069000FCC0DC015A96AD90BD90CD90DC905D978A
:1006A00052962D913D914D915C915597E985FA8532
:1006B000CF01A0E0B0E08A0D9B1DAC1DBD1D281729
:1006C00039074A075B0740F4B9016A197B097A8741
:1006D0006987672B09F4DCC0D301ED91FC91119778
:1006E000208931893A8329835E966D917C915F9749
:1006F0007C876B87C901A0E0B0E08B839C83AD83CE
:10070000BE83672BE1F5F3010088F189E02DFC87BA
:10071000EB87EF2B39F4A114B104C104D10409F41F
:10072000B7C0B3C0A114B104C104D10441F1860122
:1007300075012B803C804D805E80509440943094B5
:100740002094211C311C411C511C10C06B857C85E0
:10075000D3018D919C910E94D7029C878B87892B16
:1007600009F493C0E20CF31C041D151D6B817C8100
:100770008D819E81E616F7060807190738F7C6012E
:10078000B5012B813C814D815E810E9441172B0177
:1007900089849A84D301ED91FC91A980BA80A41830
:1007A000B5088A149B0408F45401C080D1807201FA
:1007B00000E010E086899789A08DB18DE80EF91EC2
:1007C0000A1F1B1FEB85FC853297BF0180E090E07C
:1007D0003296FC87EB872B813C814D815E810E94A4
:1007E000EE16E60EF71E081F191FD601ED91FC91BB
:1007F00095014F815885C801B7010995882361F19A
:100800008A189B08C501A0E0B0E0F301228D338D6A
:10081000448D558D280F391F4A1F5B1FD3015A96EF
:100820002D933D934D935C935D97C501840D951D6C
:10083000E981FA818E179F07B0F06B857C858D91D9
:100840009C910E94D7029C878B87892B51F4D301FE
:100850005F961C921E925E9749855A8548195909E0
:1008600019C0442455242B853C85F301378F268FEE
:100870008114910439F06F8178856A0D7B1D78872A
:100880006F8388CF49855A8505C04FEF5FEF02C05F
:1008900040E050E0CA012C960FB6F894DEBF0FBEC0
:1008A000CDBFCF91DF911F910F91FF90EF90DF901F
:1008B000CF90BF90AF909F908F907F906F905F9000
:1008C0004F903F902F900895CF93DF93FC01EB0161
:1008D0000097C9F161157105B1F1828D938DA48DD9
:1008E000B58D413051F0413018F0423061F50AC009
:1008F000288139814A815B8111C0288139814A81EF
:100900005B8108C0288139814A815B818289938912
:10091000A489B589280F391F4A1F5B1F82899389D3
:10092000A489B58982179307A407B50760F0228FC1
:10093000338F448F558F178E168E288339834A83C1
:100940005B8381E001C080E0DF91CF910895FC01DD
:10095000009711F0118210820895FC01009711F4A4
:1009600080E00895138E128E81E008952F923F92B9
:100970004F925F926F927F928F929F92AF92BF92AF
:10098000CF92DF92EF92FF920F931F93DF93CF935B
:10099000CDB7DEB7A9970FB6F894DEBF0FBECDBFB7
:1009A0003C012B01009709F44AC06115710509F457
:1009B00046C0FC0180899189892B09F040C0228DB5
:1009C000338DA081B1811097B9F1ED91FC91119710
:1009D00022803380AE014F5F5F4F89E0FA011192B0
:1009E0008A95E9F73C832B8352966D917D918D9189
:1009F0009C91559756960D911C915797061B170B76
:100A00006A012EE0E22E22E0F22E20E230E0AE017A
:100A1000465F5F4FF1010995882371F08D809E80BC
:100A2000AF80B88481149104A104B10429F021C0DD
:100A3000F20180818823A9F5F301138E128E80E0E4
:100A4000A9960FB6F894DEBF0FBECDBFCF91DF9150
:100A50001F910F91FF90EF90DF90CF90BF90AF90DC
:100A60009F908F907F906F905F904F903F902F90CE
:100A7000089588E1F20111928A95E9F709856201EA
:100A80009BE3E92E92E0F92E10E020E230E0AE0187
:100A9000465F5F4FC501B401F1010995882361F2FA
:100AA000C7CFF301828D938D0196938F828F81E062
:100AB000C7CFFB01892B61F06115710549F088E111
:100AC000DB011D928A95E9F780E1858781E0089531
:100AD00080E008952F923F924F925F926F927F92A3
:100AE0008F929F92AF92BF92CF92DF92EF92FF923E
:100AF0000F931F93DF93CF93CDB7DEB7E0970FB679
:100B0000F894DEBF0FBECDBF6C01009709F490C111
:100B1000ABC1EEE7F1E08AE1DF011D928A95E9F7CA
:100B2000D0927F01C0927E01D60119962D913D9100
:100B30004D915C911C9719E0220F331F441F551FE4
:100B40001A95D1F72AA33BA34CA35DA3CA01B9010F
:100B5000655F7F4F8F4F9F4FED91FC9129E130E012
:100B6000AE014F5F5F4F0995882309F484C1A980C6
:100B70004A80BB81BEA30C81FD801E813F815884C9
:100B800069847A849D8580E02C85E22FF0E0E82B53
:100B9000F92B8E883F88288DE98C309709F46BC13A
:100BA000432D50E060E070E0962F852F742F66276C
:100BB00069A77AA78BA79CA7822F90E0A0E0B0E05E
:100BC000BC015527442789A59AA5ABA5BCA5842BB4
:100BD000952BA62BB72B482D50E060E070E0842BBE
:100BE000952BA62BB72B89A79AA7ABA7BCA78E2DB1
:100BF00090E0A0E0B0E0782F66275527442789A52C
:100C00009AA5ABA5BCA5842B952BA62BB72B89A7A2
:100C10009AA7ABA7BCA70097A105B10589F4972DAA
:100C200080E0662D70E0682B792B6115710509F461
:100C300022C1CB01A0E0B0E089A79AA7ABA7BCA7CF
:100C4000942D80E02A2C3324282A392A952D80E0FF
:100C5000A32FB0E0A82BB92BB8A7AFA39F2D80E09E
:100C6000202F30E0822B932B9C0140E050E02A8F14
:100C70003B8F4C8F5D8FBF0180E090E0212F30E0F3
:100C800040E050E00E94EE166E8F7F8F88A399A3FC
:100C9000E9A4FAA40BA51CA54A8D5B8D6C8D7D8DF6
:100CA000E41AF50A060B170B6E8D7F8D88A199A1AA
:100CB000E61AF70A080B190BC10101972FA138A5F5
:100CC000B5E0220F331FBA95E1F7820F931FB101F0
:100CD0000E941A1780E090E0E61AF70A080B190B39
:100CE0007EA1272F30E040E050E0C801B7010E940C
:100CF000411729013A01D301C201855F9F40A040FD
:100D0000B0408050904FA040B04008F0B4C086E0A2
:100D1000D60118968C93A0E88A2EA1E09A2E88E13D
:100D2000F40111928A95E9F75101CC24DD2469A5DB
:100D30007AA58BA59CA5A60195010E94EE1660934D
:100D40008001709381018093820190938301C60199
:100D5000B5012A8D3B8D4C8D5D8D0E94EE167B0179
:100D60008C012AA13BA14CA15DA1E20EF31E041F40
:100D7000151FE0928401F092850100938601109383
:100D8000870142E050E060E070E0440E551E661EB0
:100D9000771E440C551C661C771C409288015092AB
:100DA000890160928A0170928B0130928D012092AC
:100DB0008C015EA1852F90E0BC01269EC001279E7C
:100DC000900D369E900D112490938F0180938E018B
:100DD0006E8D7F8D88A199A1A60195010E94EE16C6
:100DE0006E0D7F1D801F911F609390017093910184
:100DF0008093920190939301AFA1B8A59D0140E02B
:100E000050E0E5E0220F331F441F551FEA95D1F74C
:100E1000620F731F841F951F609394017093950157
:100E2000809396019093970194012250304002C024
:100E300020E030E0C901E0960FB6F894DEBF0FBEA7
:100E4000CDBFCF91DF911F910F91FF90EF90DF9079
:100E5000CF90BF90AF909F908F907F906F905F905A
:100E60004F903F902F90089580917E0190917F0147
:100E7000892BF1F64ECE10927F0110927E01D8CFD1
:100E8000CF93DF939C01DB01009729F16115710578
:100E900011F11D968C911D9784FF1DC08091260134
:100EA00090912701892B19F4E6E2F1E008C08091C6
:100EB000420190914301892B71F4E2E4F1E0EF01EA
:100EC000229688E10D9009928150E1F731832083C9
:100ED000138E128E02C0E0E0F0E0CF01DF91CF91DF
:100EE00008952F923F924F925F926F927F928F92CE
:100EF0009F92AF92BF92CF92DF92EF92FF920F93A9
:100F00001F93DF93CF93CDB7DEB72A970FB6F89430
:100F1000DEBF0FBECDBF4C017C836B831A010097EF
:100F200009F4DEC0672B09F4DBC04115510509F453
:100F3000D7C0DC015A96ED90FD900D911C915D9704
:100F400080E09EEFAFEFBFEFE822F9220A231B23D8
:100F5000D4015A96ED92FD920D931C935D97529693
:100F60002D913D914D915C9155972E153F05400770
:100F7000510708F4B8C0C101A0E0B0E08E0D9F1D7C
:100F8000A01FB11F281739074A075B0728F419016A
:100F90002E183F0809F4A7C0D401ED91FC911197D8
:100FA000208931893A8329835E968D919C915F9740
:100FB0009A878987290166247724892BD9F5509649
:100FC0000D90BC91A02DBA87A987AB2B39F4E11401
:100FD000F1040105110509F486C082C0E114F10491
:100FE0000105110539F15701680188279927DC01AE
:100FF00084199509A609B7098D839E83AF83B887A5
:1010000014C069857A85D4018D919C910E94D70284
:101010009A878987892B09F463C08D819E81AF816E
:10102000B885A80EB91ECA1EDB1EA414B504C604DA
:10103000D70438F7510191E0291692E0390618F0EB
:10104000A12C82E0B82EC801B701A30192010E9431
:1010500041177B0129813A81261B370B65012A152F
:101060003B0508F4690100E010E0D401ED91FC912A
:1010700086899789A08DB18DE80EF91E0A1F1B1F66
:10108000E985FA853297BF0180E090E03296FA87D1
:10109000E987A30192010E94EE16E60EF71E081FD3
:1010A000191F96014B815C81C801B7010E946E0C2B
:1010B000892BC9F0960140E050E0F401828D938DB8
:1010C000A48DB58D820F931FA41FB51F828F938FA0
:1010D000A48FB58F29853A85378F268FA50105C046
:1010E0004FEF5FEF02C040E050E0CA012A960FB612
:1010F000F894DEBF0FBECDBFCF91DF911F910F914E
:10110000FF90EF90DF90CF90BF90AF909F908F9027
:101110007F906F905F904F903F902F900895CF9366
:10112000DF939C01FB01009731F06115710519F007
:10113000858584FF2CC060E08CE790E003C060E010
:1011400088E690E00E94D70C20E030E0C901DF91F2
:10115000CF910895C0E6D1E0DF0188E10D900992BA
:101160008150E1F730935F0120935E011092780186
:101170001092790110927A0110927B0186859785F1
:1011800090937D0180937C012EE531E0DFCF80914B
:101190005E0190915F01892B91F6DCCFFC010097F5
:1011A00011F480E00895108681E008958F929F9257
:1011B000AF92BF92CF92DF92EF92FF920F93DF93A5
:1011C000CF93CDB7DEB760970FB6F894DEBF0FBEF2
:1011D000CDBF7C016B015A014901009709F493C00E
:1011E0006115710509F48FC004300CF08CC007FD47
:1011F0001DC0602F772767FD7095E4E0660F771FAD
:10120000EA95E1F762547E4F882777FD8095982F05
:1012100020E130E0AE014F5F5F4FF7010995882371
:1012200009F471C08D81882309F46DC08091A001FB
:10123000882309F068C07CC08D818093A0012A8535
:1012400030E040E050E0542F432F322F22278B858F
:1012500090E0A0E0B0E0DC0199278827282B392B0B
:101260004A2B5B2B898590E0A0E0B0E0282B392B3E
:101270004A2B5B2B8C8590E0A0E0B0E0B82FAA272A
:1012800099278827282B392B4A2B5B2B2093A101E8
:101290003093A2014093A3015093A4012E8530E026
:1012A00040E050E0542F432F322F22278F8590E0CB
:1012B000A0E0B0E0DC0199278827282B392B4A2BA6
:1012C0005B2B8D8590E0A0E0B0E0282B392B4A2BDA
:1012D0005B2B888990E0A0E0B0E0B82FAA2799277F
:1012E0008827282B392B4A2B5B2B2093A501309381
:1012F000A6014093A7015093A80103C08FEF8093EC
:10130000A0019F0102C020E030E0C90160960FB645
:10131000F894DEBF0FBECDBFCF91DF910F91FF904C
:10132000EF90DF90CF90BF90AF909F908F900895F7
:10133000E8E9F1E081E1DF011D928A95E9F7F09299
:101340009901E0929801D0929B01C0929A01B092CB
:101350009D01A0929C0190929F0180929E0107FFA7
:101360006BCFCCCF81E0089581E00895282F8FEFD7
:101370008EBD0DB407FEFDCF8DB58F778DBD8EB5BB
:10138000822F80648EBD0DB407FEFDCF8DB58F77A3
:101390008DBD872F9927AA27BB278EBD0DB407FEC9
:1013A000FDCF8DB58F778DBDCB01AA27BB278EBD15
:1013B0000DB407FEFDCF8DB58F778DBDBB27A72F51
:1013C000962F852F8EBD0DB407FEFDCF8DB58F777F
:1013D0008DBD4EBD0DB407FEFDCF8DB58F778DBD94
:1013E000222311F08FEF01C085E98EBD0DB407FEF9
:1013F000FDCF8DB58F778DBD90E02FEF2EBD0DB455
:1014000007FEFDCF8DB58F778DBD8EB58F3F19F45B
:101410009F5F9A3099F70895CF93DF93239A259A87
:10142000229A24982A9A83E58CBD8DB58E7F8DBD36
:1014300020E030E09FEF9EBD0DB407FEFDCF8DB5DF
:101440008F778DBD8EB52F5F3F4F2A30310599F7CD
:101450002A98C0E0D0E040E050E060E070E080E03A
:101460000E94B609813031F081E0CF3FD807E1F02A
:101470002196F1CFC0E0D0E040E050E060E070E0C5
:1014800081E00E94B60980FF06C08FE7CF3FD807F2
:1014900059F02196F1CF40E052E060E070E080E149
:1014A0000E94B609882319F02A9A80E008C02A9A77
:1014B0008CB58C7F8CBD8DB581608DBD81E0DF9159
:1014C000CF9108958F929F92AF92BF92DF92EF9249
:1014D000FF920F931F93CF93DF937B018C015A01EF
:1014E000E901DD24DA94812C42E0942E5EC02A9832
:1014F000B801A70140705E7F81E10E94B609882390
:1015000019F02A9A80E055C0DEBC0DB407FEFDCF6D
:101510008DB58F778DBD8EB58E3FB1F7A701517018
:10152000B401641B750BC617D70708F4BE01FB0195
:10153000E40FF51F20E030E0DEBC0DB407FEFDCF68
:101540008DB58F778DBD8EB52417350730F02E17EA
:101550003F0718F4D5018D935D012F5F3F4FB2E037
:1015600020303B0749F7DEBC0DB407FEFDCF8DB53B
:101570008F778DBD8EB5DEBC0DB407FEFDCF8DB56A
:101580008F778DBD8EB52A9ADEBC0DB407FEFDCFD8
:101590008DB58F778DBD8EB5C61BD70BCB01A0E067
:1015A000B0E0E80EF91E0A1F1B1F209709F09FCF1D
:1015B00081E0DF91CF911F910F91FF90EF90DF902D
:1015C000BF90AF909F908F9008952091000130912F
:1015D00001019FEF0AC09EBD0DB407FEFDCF8DB582
:1015E0008F778DBD8EB52F5F3F4F82E0203038075B
:1015F00090F38FEF8EBD0DB407FEFDCF8DB58F77C5
:101600008DBD8EB58FEF8EBD0DB407FEFDCF8DB5B0
:101610008F778DBD8EB52A9A8FEF8EBD0DB407FEE4
:10162000FDCF8DB58F778DBD8EB58FEF9FEF9093EA
:1016300001018093000108952F923F924F925F9293
:101640006F927F928F929F92AF92BF92CF92DF92D2
:10165000EF92FF920F931F93DF93CF93CDB7DEB737
:101660002C970FB6F894DEBF0FBECDBF4B015C01C7
:101670001A013C872B872801FE82ED82D886CF8213
:101680004115510509F4DAC02115310509F4D6C018
:101690000217130708F4D2C0EF2809F4CFC02A9824
:1016A000309521953F4F3A87298784011170D501E4
:1016B000C40180709E7F89839A83AB83BC83AC0115
:1016C000BD0181E10E94B609882311F02A9AB6C0B3
:1016D0009FEF9EBD0DB407FEFDCF8DB58F778DBDFD
:1016E0008EB58E3FA9F720E030E00BC0AFEFAEBD66
:1016F0000DB407FEFDCF8DB58F778DBD8EB52F5FF5
:101700003F4F2017310790F3E12C52E0F52EE01AFD
:10171000F10A3701EB85FC856E1A7F0A6201CE1A49
:10172000DF0A00E012E00E191F092B853C85E21646
:10173000F30648F14216530630F1F10120E030E0A3
:101740000CC08FEF8EBD0DB407FEFDCF8DB58F772A
:101750008DBD8EB581932F5F3F4FAB85BC852A171A
:101760003B0778F3A80160E070E0480D591D6A1D41
:101770007B1D2F813885C101ED81FE81099588236C
:1017800021F491E026C090E024C02B853C85E21A2C
:10179000F30A421A530A61147104A9F389859A85E0
:1017A000680E791EC80ED91E020F131FC9018C0DB9
:1017B0009D1D892B09F0B9CFE6CFAFEFAEBD0DB4BB
:1017C00007FEFDCF8DB58F778DBD8EB50894E108EE
:1017D000F108E114F10489F7BFEFBEBD0DB407FEB7
:1017E000FDCF8DB58F778DBD8EB5EFEFEEBD0DB40E
:1017F00007FEFDCF8DB58F778DBD8EB52B853C85D2
:101800004216530678F0992369F489809A80AB8058
:10181000BC8080E092E0A0E0B0E0880E991EAA1E95
:10182000BB1E43CF2A9A8FEF8EBD0DB407FEFDCFAE
:101830008DB58F778DBD8EB581E001C080E02C968F
:101840000FB6F894DEBF0FBECDBFCF91DF911F91D1
:101850000F91FF90EF90DF90CF90BF90AF909F904F
:101860008F907F906F905F904F903F902F90089552
:10187000FC0120910001309101014FEF2F3F34070F
:1018800031F460E086E890E00E94D70CFFCFCB01F6
:10189000820F931F8150924020F060E072E0621B43
:1018A000730B20E030E04FEF14C04EBD0DB407FEC7
:1018B000FDCF8DB58F778DBD8EB581938091000161
:1018C00090910101019690930101809300012F5F97
:1018D0003F4F2617370748F3CB010895CF92DF9289
:1018E000EF92FF920F931F93CF93DF937B018C01B5
:1018F0006A0180910001909101018F5F9F4F31F04B
:1019000060E08BE890E00E94D70CFFCFE90182E015
:101910002130380710F0C0E0D2E02A9880E09EEF36
:10192000AFEFBFEFE822F9220A231B23B801A7017A
:1019300081E10E94B609882321F02A9AC0E0D0E014
:101940002CC09FEF9EBD0DB407FEFDCF8DB58F77E8
:101950008DBD8EB58E3FB1F710920101109200013E
:101960002FEF14C02EBD0DB407FEFDCF8DB58F77C0
:101970008DBD8EB5D6018D936D0180910001909142
:101980000101019690930101809300018091000173
:10199000909101018C179D0728F3CE01DF91CF9123
:1019A0001F910F91FF90EF90DF90CF9008950F93CC
:1019B0001F93CF93DF93EC01062F10E005C088EE54
:1019C00093E00E94F0121F5FFE01E10FF11D649190
:1019D0006623A9F7002351F06AE088EE93E00E94A5
:1019E000F8126DE088EE93E00E94F812DF91CF913B
:1019F0001F910F9108951F920F920FB60F9211240D
:101A00002F933F934F938F939F93AF93BF93EF93F6
:101A1000FF93E091A901F091AA01309709F4A8C0C1
:101A20002091AF033091B0038091B1039091B20344
:101A30002817390709F047C08091B4038823B9F10A
:101A40008091AB039091AC032BEA32E041E08B3AFA
:101A5000940749F43093AC032093AB039093AE0307
:101A60008093AD030AC08BEA91E09093AC0380931E
:101A7000AB033093AE032093AD038091AB03909101
:101A8000AC039093B0038093AF0380509F4F90932B
:101A9000B2038093B1031092B4038091B3038823FF
:101AA00091F480916F00846080936F000CC08189F5
:101AB0009289A389B4890196A11DB11D818B928B56
:101AC000A38BB48B55C05A985C985B9A5B985C9AD0
:101AD0005B9A5B985B9A5B985B9A5B988781803195
:101AE00019F5E091AF03F091B0038181805890E047
:101AF00087FF02C05C9A01C05C985B9A5B989F5F0D
:101B0000983011F0880FF4CF908180E097FF02C0E9
:101B10005C9A01C05C985B9A5B988F5F843011F08F
:101B2000990FF4CF32961DC08830F9F4E091AF03DD
:101B3000F091B003908180E097FF02C05C9A01C0F1
:101B40005C985B9A5B988F5F883011F0990FF4CFA7
:101B50005B9A5B985B9A5B985B9A5B985B9A5B98E5
:101B60003196F093B003E093AF035A9A5D985D9A73
:101B7000FF91EF91BF91AF919F918F914F913F91C5
:101B80002F910F900FBE0F901F90189508950895F4
:101B9000DC015696ED91FC9157976289738984898F
:101BA000958908959A01AB0160E074E284EF90E0BA
:101BB0000E94411730938900209388000895CF93A5
:101BC000DF93EC0180916F008D7F80936F008D8992
:101BD000882319F00E94E50A1D8AE091A901F0917D
:101BE000AA01108A1092AA011092A901DF91CF9147
:101BF00008950F931F93DF93CF9300D000D0CDB7FC
:101C0000DEB78C01407049835A836B837C83DC018F
:101C100050968C91882351F0F894F8018589882397
:101C200029F00E94E50AD80155961C9240E0BE01B9
:101C30006F5F7F4FF801868997890E946404D801FD
:101C40005696ED91FC91579782899389A489B5891D
:101C500029813A814B815C81821B930BA40BB50BCC
:101C6000F80180879187A287B38778940F900F90AF
:101C70000F900F90CF91DF911F910F910895CF9208
:101C8000DF92EF92FF920F931F93DF93CF93CDB725
:101C9000DEB728970FB6F894DEBF0FBECDBF8C011C
:101CA0006B0144E050E07E010894E11CF11CB70197
:101CB000C6010E942103049709F0F0C044E050E0FF
:101CC00062E071E0C7010E94D116009709F0E6C0FA
:101CD000F5C044E050E067E071E0CE0105960E9457
:101CE000D116009709F0DAC0F2C044E050E06CE091
:101CF00071E0C7010E94D116009709F0CFC0F0C073
:101D0000542F432F322F22278081280F311D411D50
:101D1000511D3197EC17FD0799F7F8012487358796
:101D200046875787203131054105510509F0B6C076
:101D300048E050E0BE016F5F7F4FC6010E94210363
:101D4000089709F0ABC08A8190E0A0E0B0E0BA2F1C
:101D5000A92F982F88272981820F911DA11DB11DC0
:101D60000197A105B10521F061E088EA90E084C007
:101D70008C8190E0A0E0B0E02227382F492F5A2F25
:101D80008B81280F311D411D511D23303105410527
:101D9000510508F083C0F8012083FE013896BE018A
:101DA0006C5F7F4F542F432F322F22278081280FC3
:101DB000311D411D511D3197E617F70799F7F801BD
:101DC000218332834383548348E050E0BE016F5F38
:101DD0007F4FC6010E942103089709F05FC08E81E2
:101DE00090E0A0E0B0E0BA2FA92F982F88272D818E
:101DF000820F911DA11DB11DF801968385838885F1
:101E000090E0A0E0B0E02227382F492F5A2F8F8191
:101E1000280F311D411D511D21313105410551054D
:101E200008F03CC0278381819281A381B4818332F1
:101E3000F6E59F07F0E0AF07F0E0BF0718F02930A4
:101E400040F00CC081589E43A040B04050F0293073
:101E500040F0FF24F8018081823020F0FF24F394C9
:101E600001C0FF2461E087EA90E00E94D70CFF20C8
:101E700031F061E081E990E00E94D70C0FC0F801D9
:101E80001086118612861386D78AC68A118A128A0C
:101E9000138A148A108A158A81E001C080E028968E
:101EA0000FB6F894DEBF0FBECDBFCF91DF911F916B
:101EB0000F91FF90EF90DF90CF90089548E050E0B1
:101EC000B701C6010E942103089741F702CF44E001
:101ED00050E0B701C6010E9421030497F9F605CF2F
:101EE000F801148615861686178644E050E0B7017F
:101EF000C6010E942103049789F6F80124853585DF
:101F000046855785FE013496FBCEAF92BF92CF92A5
:101F1000DF92EF92FF920F931F93DF93CF9300D046
:101F200000D00F92CDB7DEB76C015B01F42EE52E29
:101F3000FC0180859185A285B3850097A105B10537
:101F4000D1F544E050E08E010F5F1F4FB801868944
:101F500097890E942103049709F0F5C01D8244E08F
:101F600050E0B801D60156968D919C9157970E94EA
:101F70002103049709F0E7C0F60110861186128646
:101F80001386FE01349620E030E040E050E0542F0C
:101F9000432F322F22278081280F311D411D511DD3
:101FA0003197EC17FD0799F7D60118962D933D93BD
:101FB0004D935C931B978F2D9E2D9C017901B2E070
:101FC00021303B0718F0E12C72E0F72EF601208556
:101FD000318542855385C701A0E0B0E02817390755
:101FE0004A075B0708F47901D6015696ED91FC91FA
:101FF0005797828D938DA48DB58D9170A070B07020
:102000000097A105B105D1F4D60155968C9188238E
:10201000A9F4A701B501CF010E9471078C018E15AB
:102020009F0541F060E082EE90E00E94D70C0E9494
:10203000E50A8BC081E0F601858B73C0D601559609
:102040008C91882309F463C0B701C5010E94380C44
:102050005C018E159F0539F060E08CED90E00E94E8
:10206000D70C0E94E50AD6015696ED91FC91579740
:10207000C501A0E0B0E0228D338D448D558D820FD7
:10208000931FA41FB51F828F938FA48FB58F91705C
:10209000A070B0700097A105B10509F041C00E9481
:1020A000E50AF601158A06891789D801ED90FC909A
:1020B0001197F7012089318940E050E05A966D91DF
:1020C0007D918D919C915D970E94411761157105DD
:1020D0008105910529F5D8015E966D917C915F97F8
:1020E000C7010E94D702F801978F868F892BC1F410
:1020F000D6015696ED91FC915797178E168E61E09A
:1021000082EC90E00E94D70C0FEF1FEF1EC0A701DA
:10211000B501CF010E9421038E159F05A1F401C0D6
:102120007501970140E050E0F60180859185A28518
:10213000B385821B930BA40BB50B80879187A28775
:10214000B387870102C000E010E0C8010F900F9034
:102150000F900F900F90CF91DF911F910F91FF90F3
:10216000EF90DF90CF90BF90AF900895CF92DF9225
:10217000EF92FF920F931F93CF93DF93EC01C980EF
:10218000DA80EB80FC809093AA018093A9010BEA8E
:1021900011E01093B0030093AF0342E050E0B801A8
:1021A0000E94850F892B09F451C08091AF03909153
:1021B000B00302969093B2038093B103EE89FF8936
:1021C000828D40E051E0481B5109B8016E5F7F4F9E
:1021D0008091A9019091AA010E94850F9C0100970E
:1021E000A9F18091B1039091B203820F931F909354
:1021F000B2038093B10340E051E06BEA72E080915A
:10220000A9019091AA010E94850F81E08093B403F7
:10221000888B1092800089E08093810060E074E2F6
:1022200084EF90E0A70196010E9441173093890046
:102230002093880081E090E090938B0080938A0047
:1022400080916F00826080936F007894DF91CF91CE
:102250001F910F91FF90EF90DF90CF9008951F9204
:102260000F920FB60F9211242F933F934F935F93CA
:102270006F937F938F939F93AF93BF93EF93FF934E
:1022800080916F008B7F80936F008091B4038823CF
:10229000F9F481E08093B30378946091AD03709179
:1022A000AE0340E051E08091A9019091AA010E9403
:1022B000850F892B31F48091A9019091AA010E9488
:1022C000DF0DF8941092B30381E08093B403789407
:1022D000FF91EF91BF91AF919F918F917F916F91FE
:1022E0005F914F913F912F910F900FBE0F901F90D4
:1022F000189587EB93E00E94F8008FEB93E00E9423
:10230000C70D08950F931F938FEB93E00E94DF0D8D
:102310006091BD037091BE0307EB13E0C8010E94FA
:10232000F900C8010E94FD001F910F910895CF93FD
:10233000DF93EC018091CF03882361F08FEB93E072
:102340000E94DF0D6091BD037091BE0387EB93E0A7
:102350000E94F90087EB93E00E94FD00BE0187EB2D
:1023600093E00E945301BC019093BE038093BD0390
:10237000009751F08FEB93E00E943F0E882321F0ED
:102380008FEB93E00E94B610DF91CF9108950E94E9
:1023900097118091CF038823E1F76091BD0370917D
:1023A000BE0387EB93E00E94F900089588EE93E066
:1023B0000E94E812882399F088EE93E00E94E512CB
:1023C0008093DA038093D80390E0A0E0B0E020E0AF
:1023D00030E0AC01BD0188EE93E00E945F142091D3
:1023E000D8031216E4F58091D903281709F441C0E7
:1023F0002093D9032A3094F4205D2093DB038EE2EE
:102400008093DC0387E58093DD0381E48093DE0322
:1024100086E58093DF031092E0031CC0822F6AE000
:102420000E940D17805D8093DB03822F6AE00E947B
:102430000D17905D9093DC038EE28093DD0387E5BA
:102440008093DE0381E48093DF0386E58093E003DD
:102450001092E1038BED93E00E9497110AC02223B2
:1024600041F48091D903882321F01092D9030E946E
:1024700082118091CF03882351F48091D80388235F
:1024800031F00E9482118BED93E00E949711089524
:102490000F931F93DF93CF93CDB7DEB72D970FB672
:1024A000F894DEBF0FBECDBF87EB93E00E94FD0026
:1024B00061E088EE90E00E94D70C8E010F5F1F4F05
:1024C000B80187EB93E00E945C01882379F487EBE5
:1024D00093E00E94FD002D960FB6F894DEBF0FBE6C
:1024E000CDBFCF91DF911F910F910895B80188EE74
:1024F00093E00E943F13E4CF40E855E260E070E0D3
:1025000088EE93E00E94EB1261E171E088EE93E0C7
:102510000E943F1361E082E00E945C1561E083E06D
:102520000E945C1561E084E00E945C1561E085E03A
:102530000E945C1561E089E00E945C1587EB93E0E6
:102540000E940502882321F461E088E391E01DC028
:1025500087EB93E00E94DA01882321F461E08AE2AC
:1025600091E013C087EB93E00E94C701882321F418
:1025700061E084E191E009C087EB93E00E94930160
:10258000882331F461E082E091E00E94D70C089545
:1025900061E085EF90E00E94D70C0E9448120895F8
:1025A0000E9422150E947C120E94D611FDCF84E267
:1025B00091E09093E9038093E8030895862F0E94A9
:1025C0004A1608950E94821608950E94631608957F
:1025D0000E9452160895CB01BA010E941116089567
:1025E000DC01ED91FC910190F081E02D09950895B9
:1025F000DC01ED91FC910190F081E02D09950895A9
:102600000F931F93CF93DF938C01EB0109C02196A9
:10261000D801ED91FC910190F081E02DC801099560
:1026200068816623A1F7DF91CF911F910F910895E3
:102630000F931F938C01DC01ED91FC910190F081CF
:10264000E02D6DE00995D801ED91FC910190F081AC
:10265000E02D6AE0C80109951F910F9108950F932D
:102660001F938C01DC01ED91FC910190F081E02D34
:102670000995C8010E9418131F910F9108950F9397
:102680001F938C010E940013C8010E9418131F9110
:102690000F9108950F931F938C01DC01ED91FC9134
:1026A0000190F081E02D0995C8010E9418131F9137
:1026B0000F9108952F923F924F925F926F927F9267
:1026C0008F929F92AF92BF92CF92DF92EF92FF9242
:1026D0000F931F93DF93CF93CDB7DEB7A0970FB6BD
:1026E000F894DEBF0FBECDBF1C016A017B0141150E
:1026F00051056105710549F4DC01ED91FC910190F2
:10270000F081E02D60E3099554C088249924540198
:10271000422E55246624772401E010E00C0F1D1F83
:10272000080D191DC701B601A30192010E944117AE
:10273000F80160830894811C911CA11CB11CC70185
:10274000B601A30192010E944117C901DA016C018F
:102750007D01C114D104E104F104F1F681E0E82E19
:10276000F12CEC0EFD1EE80CF91C3E010894611CD6
:10277000711CD501C4010197A109B1096C01C818E8
:10278000D90814C0F601EE0DFF1D60816A3010F407
:10279000605D01C0695CD101ED91FC910190F08117
:1027A000E02DC10109950894E108F1086E147F0439
:1027B00049F7A0960FB6F894DEBF0FBECDBFCF91FC
:1027C000DF911F910F91FF90EF90DF90CF90BF901E
:1027D000AF909F908F907F906F905F904F903F90C1
:1027E0002F9008952AE00E945A1308950F931F9383
:1027F0008C010E94F213C8010E9418131F910F91BF
:102800000895AB0160E070E00E94F21308950F9309
:102810001F938C01AB0160E070E00E94F213C801CD
:102820000E9418131F910F910895EF92FF920F933A
:102830001F93CF93DF93EC017A018B0177FF0FC0D9
:10284000E881F9810190F081E02D6DE20995109504
:102850000095F094E094E11CF11C011D111D2AE08B
:10286000B801A701CE010E945A13DF91CF911F91A9
:102870000F91FF90EF9008950F931F938C010E948A
:102880001514C8010E9418131F910F910895AB01F0
:10289000662757FD6095762F0E94151408950F93B3
:1028A0001F938C01AB01662757FD6095762F0E9420
:1028B0001514C8010E9418131F910F910895DC018F
:1028C0002115310541F4ED91FC910190F081E02D4D
:1028D000642F099508952A30310519F40E941514C2
:1028E00008950E945A1308950F931F938C010E941C
:1028F0005F14C8010E9418131F910F9108951F9231
:102900000F920FB60F9211242F938F939F93AF9333
:10291000BF938091EA039091EB03A091EC03B091F7
:10292000ED038050904CAF4FBF4F8093EA039093DC
:10293000EB03A093EC03B093ED0327C08091EA036F
:102940009091EB03A091EC03B091ED0380589E436E
:10295000A040B0408093EA039093EB03A093EC0374
:10296000B093ED038091EE039091EF03A091F003FB
:10297000B091F1030196A11DB11D8093EE039093D8
:10298000EF03A093F003B093F1038091EA039091D9
:10299000EB03A091EC03B091ED0381589E43A0405E
:1029A000B04060F6BF91AF919F918F912F910F90A2
:1029B0000FBE0F901F9018958FB7F8942091EE03DB
:1029C0003091EF034091F0035091F1038FBFB901B3
:1029D000CA010895EF92FF920F931F937B018C0120
:1029E0008FB7F8944091EE035091EF036091F0039C
:1029F0007091F1038FBF2FB7F8948091EE039091FF
:102A0000EF03A091F003B091F1032FBF841B950B4E
:102A1000A60BB70B8E159F05A007B10760F31F919A
:102A20000F91FF90EF900895019759F0FC01EE0F80
:102A3000FF1FEE0FFF1F32978FB7F8943197F1F712
:102A40008FBF0895789484B5826084BD84B5816019
:102A500084BD85B5826085BD85B5816085BDEEE6A6
:102A6000F0E0808181608083E1E8F0E08081826035
:102A70008083808181608083E0E8F0E080818160F4
:102A80008083E1EBF0E0808184608083E0EBF0E024
:102A9000808181608083EAE7F0E0808184608083C8
:102AA0008081826080838081816080838081806872
:102AB00080831092C1000895282F30E0C901825907
:102AC0009E4FFC019491265A3E4FF9018491882330
:102AD00081F0E82FF0E0E55BFE4FE491F0E0662343
:102AE00029F4808190958923808308958081892BA2
:102AF00080830895482F50E0CA018E579E4FFC01F5
:102B00002491CA0182599E4FFC019491465A5E4F0E
:102B1000FA0134913323C1F1222331F1233021F41E
:102B2000809180008F7705C0243031F4809180003F
:102B30008F7D8093800018C0213019F484B58F7781
:102B400004C0223021F484B58F7D84BD0DC02630B1
:102B500021F48091B0008F7705C0273029F480914F
:102B6000B0008F7D8093B000E32FF0E0E05BFE4F7C
:102B7000E491F0E0662329F4808190958923808395
:102B800008958081892B80830895482F50E0CA01E1
:102B90008E579E4FFC012491CA0182599E4FFC0121
:102BA0009491465A5E4FFA013491332319F420E090
:102BB00030E035C0222331F1233021F480918000B0
:102BC0008F7705C0243031F4809180008F7D809311
:102BD000800018C0213019F484B58F7704C02230EA
:102BE00021F484B58F7D84BD0DC0263021F4809101
:102BF000B0008F7705C0273029F48091B0008F7D19
:102C00008093B000E32FF0E0EB5AFE4FE491F0E048
:102C1000808120E030E0892311F021E030E0C9011B
:102C20000895EF92FF920F931F937B018C0122E096
:102C300030E040E050E00E946317205C3D4B404F85
:102C40005F4FCA01B901A80197010E946317C9012A
:102C5000DA010197A109B109292F3A2F4B2F5527E6
:102C600047FD5A950196A11DB11D2093C5008150C5
:102C70008093C400E1ECF0E08081806180838081FA
:102C8000886080838081806880831F910F91FF908E
:102C9000EF900895982F8091C00085FFFCCF90930E
:102CA000C60008958091F2039091F30380589F4FDE
:102CB0002091F4033091F503821B930B60E870E0E0
:102CC0000E942E1708954091F4035091F5038091CE
:102CD000F2039091F3038417950719F42FEF3FEF58
:102CE0000FC0FA01EA50FC4F2081CA01019660E84A
:102CF00070E00E942E179093F5038093F40330E068
:102D0000C90108958091F4039091F5039093F30322
:102D10008093F20308951F920F920FB60F92112421
:102D20002F933F934F935F936F937F938F939F93D3
:102D3000AF93BF93EF93FF934091C600E091F203EE
:102D4000F091F303CF01019660E870E00E942E1726
:102D50009C018091F4039091F5032817390739F00D
:102D6000EA50FC4F40833093F3032093F203FF912A
:102D7000EF91BF91AF919F918F917F916F915F91F3
:102D80004F913F912F910F900FBE0F901F9018956C
:102D9000FB01DC018D91019080190110D9F3990B91
:102DA0000895FB01DC014150504030F08D910190BD
:102DB000801919F40020B9F7881B990B0895FB01BD
:102DC000DC014150504048F001900D920020C9F7BD
:102DD00001C01D9241505040E0F70895629FD0011C
:102DE000739FF001829FE00DF11D649FE00DF11DC6
:102DF000929FF00D839FF00D749FF00D659FF00D75
:102E00009927729FB00DE11DF91F639FB00DE11D61
:102E1000F91FBD01CF011124089587FB082E062656
:102E200087FD819567FD619569D00EF4919507FC4A
:102E300081950895AA1BBB1B51E107C0AA1FBB1FA8
:102E4000A617B70710F0A61BB70B881F991F5A9536
:102E5000A9F780959095BC01CD01089597FB092EA7
:102E600007260AD077FD04D0E5DF06D000201AF44B
:102E7000709561957F4F0895F6F7909581959F4FD6
:102E80000895A1E21A2EAA1BBB1BFD010DC0AA1FAB
:102E9000BB1FEE1FFF1FA217B307E407F50720F0C3
:102EA000A21BB30BE40BF50B661F771F881F991F3E
:102EB0001A9469F760957095809590959B01AC0187
:102EC000BD01CF01089597FB092E05260ED057FDB1
:102ED00004D0D7DF0AD0001C38F4509540953095C7
:102EE00021953F4F4F4F5F4F0895F6F7909580958E
:102EF000709561957F4F8F4F9F4F0895991B79E093
:102F000004C0991F961708F0961B881F7A95C9F779
:102F100080950895EE0FFF1F0590F491E02D099420
:042F2000F894FFCF53
:102F2400FFFF52494646005741564500666D7420DE
:102F34000041756469666F6E6F2074657374210057
:062F440000000000DE1297
:00000001FF
